:100000000004001001010000D5000000D90000002C
:1000100000000000000000000000000000000000E0
:100020000000000000000000000000009905000032
:100030000000000000000000510500000105000064
:1000400045010000450100000000000045010000DE
:100050004501000045010000000000000000000014
:100060004501000045010000450100004501000078
:1000700045010000450100000000000045010000AE
:100080000000000000000000000000000000000070
:100090000000000000000000000000000000000060
:1000A0004501000045010000450100004501000038
:1000B0004501000045010000450100004501000028
:1000C000D808000000000010040000000400001028
:1000D0004002000000B5FEE700B5FEE710B50023C2
:1000E00002E01C58043310C19342FAD310BD10B57E
:1000F000031C002200E004C31C1A8C42FBD310BD79
:1001000038B50D4C0D4D05E020686168A2680C34CF
:10011000FFF7E4FFAC42F7D305E0206861680834DC
:10012000FFF7E5FF00E0064DAC42F6D300F032FBEE
:1001300000F052FBFEE7C046C0000000CC0000000B
:10014000D400000000B5FEE7F7B5304A4020D16F7B
:100150002F4B0143D167D16F80200143D16758688D
:100160002C4941240140596058688021C90001434D
:1001700059602948294964420860E02040000C5039
:10018000A020802100068901445804252C434450B6
:10019000234D2448082101272F60C167D46F802098
:1001A000C0012043D0675A681F4C8A435A605A687E
:1001B0000526114359601D4B2968186826602B6875
:1001C000002B21D000F00CFBE12105094902281C7D
:1001D00000F006FB164BFF22013820621A601868F7
:1001E000216A1B68C0190193CB19E12149025943C7
:1001F000684300F0F5FA019AD343C0180D4B18601C
:10020000A66023681F432760F7BDC04604800440F2
:1002100000800440FFFBFFFF0400FFFF00C0004020
:100220009480044004E100E000400640000000101B
:10023000F0800440F480044000B5A0231B06042293
:100240008821002800D18A2189015A5000BD000070
:1002500000B5044B9A68510701D5D86101E001202F
:10026000404200BD0040064000B5044B9A68D107EB
:1002700001D5586901E00120404200BD0040064020
:1002800010B5041C08E000F03EFA2078FFF7E0FF0C
:1002900023789842F7D101342378002BF5D110BD93
:1002A000F7B50025124E2F1CFFF7DEFF041E12DBF0
:1002B000002D05D10F48FFF7E3FF0F48FFF7E0FFE0
:1002C0000D2C01D10B4802E001A804704770FFF724
:1002D000D7FF0A4D08E0002D02D0013D002D03D1CB
:1002E000301CFFF7CDFF002500F00DFADCE7C0461B
:1002F0006C0800009808000054080000F30100009A
:1003000008B50120FFF798FFFA20400000F0F8F947
:100310000020FFF791FFFA20400000F0F1F9F0E72C
:1003200008B5FFF711FF00F0D7F9012006490A22AE
:1003300000F0A2F902200549142200F09DF900F016
:1003400069F9002008BDC04601030000A1020000B9
:1003500000B5031C30331A0419061143054A19432A
:10036000C0011B02194310180023C1500433802B15
:10037000FBD100BD04000010704700B5002901D179
:1003800006E0181C8368002BFBD1816048608B60FD
:1003900000BD00B58368002B07D09A688260002AF0
:1003A00000D0506000225A609A60181C00BD00B551
:1003B0000DE088420BD142688368002A00D0936028
:1003C000002B00D05A6000234360836002E0806805
:1003D0000028EED100BD38B50D1C00E0201C84685B
:1003E000A847002CFAD138BD10B5064A064B0720A5
:1003F00004211468844314601C698C431C6130BF61
:10040000F7E7C0460000024000ED00E070B50028AC
:1004100016DAC0B20F230340083B134A9B089B0027
:100420009B18032210409040FF225D68141C8440FA
:100430008901A5430A408240281C1043586011E0FE
:1004400003248208094B2040C032A0409200FF24C0
:10045000D558261C86408901B5430C408440281C91
:100460002043D05070BDC04618ED00E000E100E030
:1004700010B50369011C002B0DD1094C201C303034
:10048000FFF795FF011E08D00123201C0B731030CD
:10049000FFF773FF01E0013B0361002010BDC04680
:1004A0008401001010B5144CE36D002B06D000231E
:1004B000201CE36530301149FFF78DFFE16800290A
:1004C00011D00B7B012B05D0002B02D0022B04D0C6
:1004D00008E0FEE7201C103001E0201C3030FFF760
:1004E0004CFF00E0FEE7044C201C1030FFF751FFEA
:1004F000002800D0E06010BD8401001071040000ED
:1005000000B5104B104A996D01319965914204D99B
:1005100000219965596D01315965DB68D96901314F
:10052000D961914204D90022DA619A6901329A6153
:10053000044B0122DA65054B8022596852050A43B3
:100540005A6000BD84010010E703000000ED00E0E8
:10055000EFF30982203AF0C244464D4656465F46C4
:10056000F0C2203A0B49C868026000B5FFF79AFF55
:1005700001BC86460749C86802681032F0CAA04626
:10058000A946B246BB46203AF0CA103282F3098827
:100590007047C046840100101B4A50601A4A91609F
:1005A00070460421084202D0EFF3098101E0EFF325
:1005B00008818A69023A1078134A106080B484B0C6
:1005C0006F46124B1A78012A14D0002A0DD0802AC7
:1005D00016D10D49C868026882F309880421704663
:1005E000084386460A4B596807E0DA685B680221CF
:1005F00011731361064B8022596852050A435A60F1
:1006000004B080BC7047C046840100108401001013
:1006100000ED00E010B500F079F8144BFA211868ED
:10062000890000F0DDF8124C013860600120404282
:100630000321FFF7EBFE0023A360052007232360BF
:1006400040428021FFF7E2FE01204042C021FFF737
:10065000DDFE02204042FF21FFF7D8FE054B80223D
:1006600012061A6080DFC046FEE7C0460000001098
:1006700010E000E000E100E070B5154C4301E41823
:10068000151C0E1CFFF764FE031C4033236001227F
:10069000002322736360A3606561036643670D4DA9
:1006A00080235B04C3672B6D4266022282668667E5
:1006B000002B03D160302060EC6004E0281C103077
:1006C000211CFFF75AFE2B6D01332B6570BDC04610
:1006D000E40100108401001010B5074C201C1030FC
:1006E000FFF74AFE201C3030FFF746FE002003498A
:1006F0000122FFF7C1FF10BD84010010E9030000D3
:1007000000DFC046704701DFC046704770B51D4D21
:1007100000206B6ADB051B0F013B0E2B02D81A4A27
:100720009B009858696A2A6F0326164B3240174C73
:10073000022A0CD0B24212D0012A03D11B6C1E40F7
:10074000022E01D0124B00E00023236012E01F2391
:1007500019404900023100F043F820600AE0196CAA
:100760000A40022AF0D09B681F2009491840013036
:1007700041432160054CA96F206800F031F82060EA
:1007800070BDC046008004409C08000000000010BE
:10079000001BB70010B50D4A0D48D16F0D4B01433A
:1007A000D16700221A6401225A64101C5C6C09494A
:1007B00001220442FAD0002008674A67596F1142AB
:1007C000FCD0044B01229A6710BDC046048004404F
:1007D000800004000080044008B5FFF7A1FD08BDBB
:1007E000002931D00122D207030901E009011209D1
:1007F0009942FBD9430801E0490052089942FBD9CC
:1008000000E04908401A07D35241FAD30146104686
:10081000704749084018F7D29218FAD34018014699
:1008200010467047CB0F00D04942021000D540421D
:10083000534008B5FFF7D4FF0CBC521000D3404220
:10084000002A00D549421847F446002000F001F87C
:1008500060477047596561682E2049742773207975
:100860006F7572207475726E2E0D0A0054686520C3
:10087000717569636B2062726F776E20666F782086
:100880006A756D7073206F76657220746865206C70
:10089000617A7920646F672E0D0A000020A107009D
:1008A00000350C00E0C81000C05C1500006A18009C
:1008B00040771B0080841E00C0912100009F24000F
:1008C00040AC2700E032290020402C00604D2F0072
:0808D00000D4300040E13300C8
:0408D800001BB7004A
:0400000300000101F7
:00000001FF
